:100000000C9446000C9465000C9465000C946500FB
:100010000C9465000C9465000C9465000C946500CC
:100020000C9465000C946E000C9465000C946500B3
:100030000C9465000C9465000C9465000C946500AC
:100040000C9465000C9465000C9465000C9465009C
:100050000C9465000C9465000C9465000C9465008C
:100060000C9465000C9465000C9465000C9465007C
:100070000C9465000C9465000C9458060C94650073
:100080000C941B060C944E030C94650011241FBEA7
:10009000CFEFD0E1DEBFCDBF11E0A0E0B1E0E8ECF2
:1000A000FDE000E00BBF02C007900D92A831B10740
:1000B000D9F712E0A8E1B1E001C01D92A83FB10755
:1000C000E1F70E94CA000C94E2060C9400008BE059
:1000D00085BD89EF83BD80E887BF08951F920F9289
:1000E0000FB60F9211248F939F93AF93BF9380917C
:1000F000180190911901A0911A01B0911B0101966C
:10010000A11DB11D8093180190931901A0931A01AC
:10011000B0931B01BF91AF919F918F910F900FBE34
:100120000F901F9018950895FC0183899489089574
:10013000DF93CF93CDB7DEB768970FB6F894DEBFE5
:100140000FBECDBFDE011196E0E0F1E088E1019045
:100150000D928150E1F7FE0131969E01275E3F4FDF
:10016000908180919B0085FFFCCF90939C003196FD
:10017000E217F307A9F768960FB6F894DEBF0FBE33
:10018000CDBFCF91DF910895E2E6F0E08081805805
:1001900080830895EF92FF920F931F93F8940E942B
:1001A00019030E94670085E08093230260E070E0FD
:1001B00080E090E00E942B030E94BA057894809121
:1001C0006100806880936100809162008068809304
:1001D000620082E3E82EF12C00E117E220E030E03B
:1001E00040E050E060E070E088E990E00E940701A4
:1001F00008EE13E021E030E040E050E060E070E025
:1002000084EC90E00E9407010E94FF01FDCFCF9295
:10021000DF92EF92FF920F931F93CF93DF93EC0146
:100220006B01A0E0B0E09A2FFD0184E0EE0FFF1F0C
:100230008A95E1F7EA0FFB1FE45EFE4F878588236E
:1002400029F09F5F1196AC30B10569F7692F70E016
:10025000FB01A4E0EE0FFF1FAA95E1F7E60FF71FE1
:10026000E45EFE4FD183C083D382C2825583448330
:1002700037832683E114F10411F4108A08C082E365
:10028000E816F10411F481E001C082E0808BFB01EB
:1002900034E0EE0FFF1F3A95E1F7E60FF71FE45E3B
:1002A000FE4FA089B0E0A851BE4F8C91982F9E0DB3
:1002B00096878F5F8C931187008781E08787F894FA
:1002C000209118013091190140911A0150911B01A0
:1002D000C801A0E0B0E0820F931FA41FB51FFB016F
:1002E00024E0EE0FFF1F2A95E1F7E60FF71FE45E0B
:1002F000FE4F82879387A487B5877894DF91CF914B
:100300001F910F91FF90EF90DF90CF900895CF92C3
:10031000DF92EF92FF920F931F93CF93DF93DC0155
:10032000EB01690120E030E0622FF90174E0EE0F8B
:10033000FF1F7A95E1F7E20FF31FE45EFE4F87851A
:10034000882331F06F5F2F5F3F4F2C30310561F70D
:10035000262F30E0F90164E0EE0FFF1F6A95E1F708
:10036000E20FF31FE45EFE4FB183A083D383C28309
:1003700055834483D782C682E114F10411F4108AB4
:1003800008C082E3E816F10411F481E001C082E0C4
:10039000808BB90194E0660F771F9A95E1F7620FA1
:1003A000731F645E7E4FEB01E889F0E0E851FE4F79
:1003B0008081982F9E0D9E878F5F80831987088785
:1003C00081E08F87209118013091190140911A0125
:1003D00050911B01C801A0E0B0E0820F931FA41F41
:1003E000B51FFB0182879387A487B587DF91CF91E3
:1003F0001F910F91FF90EF90DF90CF900895EF92B3
:10040000FF920F931F93CF93DF93F894E09018011E
:10041000F090190100911A0110911B01789410922B
:10042000EB018091EE018F5F8093EE018091EE01F0
:10043000883C49F48091ED0186958093EC011092FF
:10044000ED011092EE014FEF5FEF20E030E0F90197
:10045000A4E0EE0FFF1FAA95E1F7E20FF31FE45EA1
:10046000FE4F8785882399F08091EB018F5F809301
:10047000EB0182859385A485B585E816F9060A0700
:100480001B0728F08685851710F45685422F2F5FAD
:100490003F4F2C303105D9F64F3FB9F18091ED0136
:1004A0008F5F8093ED01842F992787FD9095EC0154
:1004B000E4E0CC0FDD1FEA95E1F7C80FD91FC45E59
:1004C000DE4FE881F9816C817D818A819B8109956C
:1004D0008E819F81892B49F41F86E889F0E0E851DD
:1004E000FE4F80818150808310C02A853B854C85DA
:1004F0005D8588859985A0E0B0E0820F931FA41FD9
:10050000B51F8A879B87AC87BD8781E0DF91CF913C
:100510001F910F91FF90EF9008959C01DB0160E027
:1005200070E0FB0144E0EE0FFF1F4A95E1F7E60F94
:10053000F71FE45EFE4F808191818217930719F5C2
:100540008785882301F1F8942091180130911901D1
:1005500040911A0150911B01CD01A0E0B0E0820F43
:10056000931FA41FB51FFB0124E0EE0FFF1F2A9568
:10057000E1F7E60FF71FE45EFE4F82879387A487BB
:10058000B587789408956F5F7F4F6C30710549F699
:100590000895AC0120E030E0F901A4E0EE0FFF1F68
:1005A000AA95E1F7E20FF31FE45EFE4F808191818F
:1005B00084179507B9F487858823A1F02091180145
:1005C0003091190140911A0150911B01CB01A0E01B
:1005D000B0E0820F931FA41FB51F82879387A48763
:1005E000B58708952F5F3F4F2C303105A9F6089548
:1005F000AC0120E030E0F901B4E0EE0FFF1FBA9546
:10060000E1F7E20FF31FE45EFE4F808191818417D2
:10061000950749F41786E089F0E0E851FE4F8081A4
:100620008150808308952F5F3F4F2C30310519F79B
:10063000089580E090E0FC0124E0EE0FFF1F2A9572
:10064000E1F7E80FF91FE45EFE4F178601968C3044
:10065000910589F7089580912302880F8160809326
:10066000720080E480937000E1E7F0E080818C7F8D
:1006700080832FEF2093730085EC8093740081E0DA
:1006800090E09093F2018093F1011092F001209399
:100690001D02109207021092060208951F920F92F7
:1006A0000FB60F920BB60F921124EF92FF920F9399
:1006B0001F932F933F934F935F936F937F938F93EA
:1006C0009F93AF93BF93EF93FF938091F10190912C
:1006D000F201817C09F4CBC08091710090E0887FA9
:1006E00090708038910561F181389105ACF48836BD
:1006F000910509F48AC0893691052CF4803691055C
:1007000009F0B3C09AC08037910509F496C08837C4
:10071000910509F0AAC079C08039910589F0813925
:1007200091052CF48838910509F09FC096C088394E
:10073000910509F492C0803A910509F096C093C0E2
:100740008091F1019091F2018034910581F48091C2
:1007500073008093F4018FEF80931D0280E890E096
:100760009093F2018093F1011092F0017CC080918E
:10077000F1019091F2018038910509F074C09091D7
:10078000F0018091F4019817A0F48091F001E82F16
:10079000F0E090917300ED50FE4F92838F5F809355
:1007A000F00190911D0280917300892780931D02B2
:1007B0005AC08091F001803111F5809173008093CF
:1007C000050290911D0280910502981719F081E0B1
:1007D00090E002C082E090E09093070280930602CE
:1007E000EE24FF2400E010E020E030E040E050E0A4
:1007F00063EF71E084E990E00E9487012EC0809150
:10080000F0018F5F8093F0012EC0809121028F5FF5
:100810008093210280911E028A3078F422E3E22E36
:10082000F12C02E310E020E030E040E050E060E036
:1008300070E083E295E00E948701809173008093CD
:10084000F30110920702109206021092F00185EC5B
:100850008093740080E490E07DC081E090E090930C
:10086000F2018093F10185ECD5C085E4D3C080917D
:10087000710090E0887F90708032910509F49CC0EF
:100880008132910554F48031910599F088319105B8
:10089000D1F0089709F0B7C00CC08033910509F476
:1008A0005EC08833910509F460C0889709F0ABC039
:1008B00011C0809108028093730085E880937400D2
:1008C00088E090E047C01092EF0180910902809388
:1008D00073003BC08091EF018131D9F485E98093A9
:1008E000740080E290E09093F2018093F101109205
:1008F0001E0280911F029091200201969093200287
:1009000080931F0260E070E08BE293E00E94C902D6
:1009100083C09091EF0180910902981750F0809167
:100920001A02809373008091EF018F5F8093EF0133
:100930000CC09091EF01E92FF0E0E85FFD4F82815C
:10094000809373009F5F9093EF0185E8809374001C
:1009500080E190E09093F2018093F1015DC080917D
:1009600021028F5F809321022CC0809121028F5F32
:100970008093210260E070E08BE293E00E94C90264
:1009800080911E028A3080F492E3E92EF12C02E37A
:1009900010E020E030E040E050E060E070E083E212
:1009A00095E00E94870106C088E290E09093F201F2
:1009B0008093F10185E82EC0809122028F5F8093A1
:1009C000220260E070E08BE293E00E94C902809115
:1009D0001E028A3080F482E3E82EF12C02E310E05C
:1009E00020E030E040E050E060E070E083E295E03D
:1009F0000E94870106C088E290E09093F201809304
:100A0000F10185E907C084E090E09093F2018093C2
:100A1000F10185E080937400FF91EF91BF91AF9158
:100A20009F918F917F916F915F914F913F912F9106
:100A30001F910F91FF90EF900F900BBE0F900FBE84
:100A40000F901F901895EF92FF920F931F93809134
:100A5000F1019091F201019771F042E3E42EF12C43
:100A600005E010E020E030E040E050E060E070E0C1
:100A700083E295E01DC01092EF0185EA8093740037
:100A800082E090E09093F2018093F10180911E0248
:100A90008F5F80931E0232E3E32EF12C00E117E218
:100AA00020E030E040E050E060E070E08BE293E076
:100AB0000E9407011F910F91FF90EF900895EF9210
:100AC000FF920F931F93582F80911E02882309F4E1
:100AD00048C080911E028A3009F443C081E03CC0C6
:100AE0008FEF80931A02DB0120E030E00DC08C9183
:100AF000F901E85FFD4F828380911A029D91892759
:100B000080931A022F5F3F4F241788F381E0809370
:100B10001E02852F90E0880F991F80930802409352
:100B200009021092EF0185EA8093740082E090E060
:100B30009093F2018093F10152E3E52EF12C05E050
:100B400010E020E030E040E050E060E070E08BE258
:100B500093E00E94070180E01F910F91FF90EF90BA
:100B600008958091F1019091F201019709F4B8CFB5
:100B700082E0F2CF1092980087E680939900EBE92B
:100B8000F0E080818D7F808388E080939A0086E00A
:100B900080939D000895AC0180919B0085FFFCCF60
:100BA00070939C0060938E021092F3021092F202F6
:100BB0006F5F7F4F7093F7026093F6026150704051
:100BC00081E090E09093F5028093F402DA0120E056
:100BD00030E007C02F5F3F4F8D91F901E257FD4F85
:100BE000808326173707B0F30895BC0180919B00DE
:100BF00087FFFCCF30919C0080919B0087FFFCCF4A
:100C000020919C00932F80E0AC01420F511D20E009
:100C100030E00CC080919B0087FFFCCF80919C004E
:100C2000FB01E20FF31F80832F5F3F4F241735072F
:100C300088F3CA0108951F920F920FB60F920BB658
:100C40000F9211242F933F938F939F93EF93FF93D2
:100C50002091F2023091F3028091F6029091F70216
:100C60002817390780F48091F2029091F302FC0179
:100C7000E257FD4F208120939C0001969093F30250
:100C80008093F20208C01092F3021092F2021092C6
:100C9000F5021092F402FF91EF919F918F913F9195
:100CA0002F910F900BBE0F900FBE0F901F901895B5
:100CB0001F920F920FB60F920BB60F921124EF9264
:100CC000FF920F931F932F933F934F935F936F93D5
:100CD0007F938F939F93AF93BF93EF93FF938091F5
:100CE0008C0290918D02892B99F481E090E0909391
:100CF0008D0280938C0220919C00922F80E0909333
:100D00008B0280938A02109289021092880243C05B
:100D10008091880290918902892B69F480918A02DE
:100D200090918B0220919C00820F911D90938B02D9
:100D300080938A0227C0E0918802F0918902809115
:100D40009C00ED5DFD4F80832091880230918902E7
:100D500080918A0290918B022817390798F010929F
:100D60008D0210928C02EE24FF2400E010E020E0BF
:100D700030E04AE852E064E272E083E990E00E94E9
:100D8000870109C080918802909189020196909311
:100D9000890280938802FF91EF91BF91AF919F915B
:100DA0008F917F916F915F914F913F912F911F9103
:100DB0000F91FF90EF900F900BBE0F900FBE0F9012
:080DC0001F901895F894FFCF75
:100DC80014601572165817051C00939FC2868C086C
:080DD800BFA208A908801D005C
:00000001FF
